:020000040800F2
:10000000501B0020CD00000801310008E10F00085E
:1000100000000000000000000000000000000000E0
:10002000000000000000000000000000D13D0008BA
:100030000000000000000000493300086943000888
:10004000DF00000800000000DF000008DF000008FB
:10005000DF000008DF000008DF000008DF00000804
:1000600000000000DF000008B9040008590500087E
:10007000DF000008DF000008DF00000800000000CB
:10008000DF0000087544000800000000DF000008E1
:10009000DF000008DF000008DF000008DF000008C4
:1000A000DF000008D53C0008DF0000088D44000890
:1000B000154500080348854600F0D6F8004800477B
:1000C000514E0008501B00200844F0470448804768
:1000D00004480047FEE7FEE7FEE7FEE7FEE7FEE72F
:1000E00019440008B500000830B50B460146002051
:1000F0002022012409E00D46D5409D4205D31D462E
:100100009540491B2546954040191546521E002D25
:10011000F1DC30BD70B500242546002801DA012449
:100120004042002901DA01254942FFF7DDFFAC42D8
:1001300000D04042002C00D0494270BDF8B50024E8
:100140002546002904DA0E46012400214042B1412F
:10015000002B04DA1E46002352420125B34100F071
:1001600052F88C4617461E46AC4203D0002540424A
:100170008D41AC46002C02D0002657429E4161467C
:100180003A46334601B0F0BD10B5202A04DB0846DC
:10019000203AD040002110BD0B46D340D04020244F
:1001A000A21A91400843194610BD03460B439B0712
:1001B00003D009E008C9121F08C0042AFAD203E0DC
:1001C0000B780370401C491C521EF9D27047D2B202
:1001D00001E00270401C491EFBD270470022F6E786
:1001E00010B513460A4604461946FFF7F0FF2046AD
:1001F00010BD0321001D401E037812021A43491E40
:10020000F9D510467047F0B51FB40646002082B0FD
:1002100005464024019100901BE0019922460F46BB
:100220003046FFF7B1FF049A059B801A994110D31D
:1002300010461946224600F029F8361A8F410197D8
:10024000224601200021009F00F020F838184D417F
:1002500000902046641E0028DFDC019B00982946A0
:10026000324607B0F0BD0000064C0125064E05E001
:10027000E36807CC2B430C3C98471034B442F7D3C7
:10028000FFF71CFFD0580008F058000810B5202ACE
:1002900004DB0146203A9140002010BD914020230C
:1002A0009C1A0346E3401943904010BDF0B51C4C26
:1002B000A0684007C00F31D1206C1B4D82B2194895
:1002C0001A4903690120DE07002E0AD08A82184BE2
:1002D000184928469A4201D2012200E000220A6011
:1002E00012E09D4306D0144D9D4306D0134D9D430F
:1002F00006D009E00A83124806E00A84114803E0A8
:100300004A84114A528BCA834103490BA162A168F6
:100310000E4A1140091DA160024908610020F0BD8C
:10032000002401400000002000010020F412002001
:1003300098080000BC0000200000014000000244BA
:10034000000001C0000002C4A0F7FF1FE8FFFF7F0C
:10035000F0B51E4F85B03D691D4C6D1C3D61266892
:10036000A468029400966C466580019021816281A8
:100370000393386A01011748091800220B461046FA
:100380001C5CFF2C04D1401C1028F9D3002A17D084
:100390001022684600F012F9386AF861401C386291
:1003A0000001012109031030884201D90020386280
:1003B000F8680949401CF8604867002005B0F0BDA6
:1003C0001022684604F018FAE6E7000098000020C2
:1003D0008458000800D0000874120020002911D0B1
:1003E0008268521882604368934200DCD21A00236C
:1003F0008361C368934201D1012343618260026932
:10040000521802610846704710B500231A4605E0ED
:10041000845C2407240FE318DBB2521C8A42F7DB0A
:100420001807000F10BD0000F0B50020174D012780
:10043000144B154C3F03E86017E0625A144EB24269
:1004400012D1EA680919521CEA604A882E69B24240
:1004500005D92A61E8614A686A61421C2A624988B2
:10046000994201D20B46A861401C0101B942E4D374
:10047000286A00011030B84201D900202862E868DB
:10048000F0BD0000FFC99A3B00D000089800002092
:10049000AA55000010B50421054800F0B0F8054841
:1004A00000218161C1610161C1600162084610BD26
:1004B00000D000089800002070B5234DE86A401C69
:1004C000E862224C20688006C00F11D02868296B92
:1004D00040182860296B28465830064600F058F826
:1004E00020206060B06900280AD00020286368726C
:1004F00020688005C00F02D001204002606070BDFE
:10050000304600F009FA12494A78A3585B085B00AC
:10051000A350F36832684E78D2180C4B0C33F2506B
:100520000A4B4A781B1DD658360C36040643D65063
:100530004978625801231A4362502863054881684C
:10054000802211438160D3E71402002000000240A2
:1005500099580008003801400B49C86A401CC8621D
:100560000A4802689204D20F05D001225203426069
:1005700000220A634A7201688903C90F02D001216F
:100580004904416070470000A802002000000240BA
:1005900010B5002910D0C26843685218934200DC9D
:1005A000D21A00234361C2608468944204D10122BC
:1005B00082618360C360C361084610BDF0B585B039
:1005C00016460D46074600F007FB0120029000206A
:1005D0000090019503A9684600F066FA00247608A9
:1005E00007E060003A5A41190023012000F0B6FAF2
:1005F000641CA642F5D800F0A7FA05B0F0BD7FB59F
:100600000D46044600F0E8FA00206A4631C203A90C
:10061000684600F049FA00F097FA04B070BD000097
:1006200006490020C861064801690422114301619E
:10063000016940221143016170470000301700201A
:1006400000200240064A0021D16106490A690223BE
:100650001A430A61486108694022104308617047E3
:10066000301700200020024010B5054B0022DA614F
:10067000044A1369012423431361018010BD000063
:10068000301700200020024010B50B4A0020D1682E
:10069000CB060A4904D5C86902231843C861102053
:1006A000D3685B0705D5CB6901242343CB610421C3
:1006B0000843D06010BD0000002002403017002029
:1006C00070B5044600F09AFA0546104E0AE0601C28
:1006D00008D0002C04D000F091FA401BA04201D9B0
:1006E000032070BDF068C007F1D1F068800601D525
:1006F0002020F060F068C00602D4F068400703D5FF
:10070000FFF7C2FF012070BD002070BD0020024035
:1007100010B50E4C0020207220710D480078002882
:1007200000D10120A070E0700120C0020921C9069B
:10073000886288620749802088620A2000F0A6F952
:1007400000F08EF96061002010BD0000C80000209C
:100750005700002000140048FEB5364D0121490223
:10076000284601F039FF00900120019040213248D5
:1007700001F032FF044601210920C902C00601F040
:100780002BFF4021284601F027FF00262B4D002893
:100790000BD0002013212A4A4901EF7803E01318F7
:1007A0005B181E75401CB842F9DB0098002802D186
:1007B00000F056F968612869012700280ED10098D9
:1007C00000280BD000F04CF96969401A1D49884295
:1007D00004DBF8020921C90688612F61002C06D1CB
:1007E000E868002803D01848018DC1840685019867
:1007F000002817D0002C17D0E86800280AD12F71E4
:100800006E711248026840218A4302606E7102686C
:100810000A430260287A002808D12879002805D1E7
:100820002F7102E0002C01D12E716E71EC6000205E
:10083000FEBD00000004004800140048C80000206D
:10084000F40C002010270000741400200038004031
:100850000A07120F01219140014201D00120704787
:10086000002070470A07120F01219140014201D078
:100870000120704700207047F8B50B051B0E254C72
:100880005B001C1909239B01E31800930523DB017E
:10089000E618012307469B020A07E5180020120FFD
:1008A0003B0003F0E3FF09060A0E12191D21282F51
:1008B0002E00FF2928D800981BE0FF2924D8009893
:1008C00008E0FF2920D8B08A18E080291CD20F2028
:1008D00080012018808E11E0802915D2A88A0DE0B1
:1008E000402911D2B08E09E040290DD20B208001A1
:1008F0000EE0808A02E0802906D2A88E1146FFF71A
:10090000B1FFF8BD802901D30020F8BD0920C00146
:100910002018EEE7F40C0020C1688268914201DAE9
:10092000501A7047914202DC4269002A02D04068A6
:10093000401A704780690028FBD000207047C268C9
:100940008168914201DA501A7047914202DC826953
:10095000002A02D04068401A704740690028FBD046
:100960000020704706490122896912030818010115
:10097000914201D3FF380138024900014018704705
:100980009800002000D00008F0B5334C4B001C1933
:100990000923DB01E5180B230246DB010020E318E5
:1009A000892A25D00EDC2C4F2C4B4E00F619F61858
:1009B000803A130003F05AFF091F1F152125292E25
:1009C000333A15008D2A3FD00CDC8A2A33D08B2A8B
:1009D00035D08C2A05D140293ADA0B208001201825
:1009E000808EF0BD992A03D0A12A01D0FE2AF8D129
:1009F00080292DDA2EE00846F0BD102928DAB08AC9
:100A0000F0BD102924DAB08EF0BD102920DA0520BF
:100A1000C00108E008291BDA0F208001DFE7082960
:100A200016DA012080022018808AF0BD80290FDAB2
:100A30003420285EF0BD80290ADAA88AF0BD40295A
:100A400006DA0D208001CAE7402901DAA88EF0BD40
:100A50000020F0BD988EF0BDF40C00204002000094
:100A600010B5074A5068074B99695468A04201D0F5
:100A700050689969044A51430914401A10BD000096
:100A80001C00002000E000E05505000031B500F03A
:100A9000B5F8009C0546601C00D0641C00F0AEF860
:100AA000401BA042FAD338BDF8B5054623480F468F
:100AB000017E012601290BD0012101762868204CF6
:100AC000012807D02046FFF7FBFD002813D030E0B7
:100AD0000220F8BD2046FFF7F3FD002829D1FFF7DB
:100AE0009FFD2046FFF7ECFD0646164801690422EB
:100AF000914301611DE00020C04338606C6812E042
:100B00002046FFF79FFD0E48FFF7DAFD06460D4829
:100B10000169022291430161002E01D03C6008E08E
:100B2000012080022418A868696880024018A04249
:100B3000E6D80248002101763046F8BD3017002083
:100B400050C3000000200240034801698022114385
:100B5000016100207047000000200240F0B51FB482
:100B600005461A480024017E16461F46012907D073
:100B7000012101761648FFF7A3FD002803D021E0EC
:100B8000022005B0F0BD012D1AD0022D18D0042589
:100B900016E0220130463946FFF7F6FA81B2019895
:100BA00062001018FFF760FD0948FFF789FD094949
:100BB0000A69520852000A61002803D1641CE4B299
:100BC000AC42E6D3014900220A76DAE7301700206A
:100BD00050C300000020024005480169090605D500
:100BE000044941600449416000207047012070477A
:100BF0000020024023016745AB89EFCD0148006822
:100C0000704700001001002002480168491C016083
:100C1000704700001001002010B50648016810223E
:100C200011430160002000F007F800F017F80020E1
:100C300010BD00000020024010B5044600F040F94D
:100C40007D21C900FFF750FA00F088FB0022214601
:100C5000501E00F025F8002010BD000008B50F4818
:100C60008169012211438161816911400091C2694A
:100C700001040A43C261C069002208400090114685
:100C8000501F00F00DF800221146901E00F008F8E9
:100C900000221146501E00F003F808BD001002406B
:100CA00010B502F05BFA10BDF8B504460068364D89
:100CB000C00354D5E8690026C00007D4E8692904B8
:100CC0000843E861E8690840012600902F48016860
:100CD000C90511D4014608688A1510430860FFF75A
:100CE0008DFF074604E0FFF789FFC01B642823D867
:100CF00026480068C005F6D5286A03210902084085
:100D00001FD062680A4082421BD0286A2A6A884340
:100D1000012109040A432A622A6A8A432A62286254
:100D2000C0070ED0FFF76AFF074607E0FFF766FF30
:100D3000C11B1748814201D90320F8BD286A8007EA
:100D4000F4D5286A032109028843616808432862B0
:100D5000002E04D0E869012109078843E861207862
:100D6000C00705D0286BA16880088000084328636D
:100D70002078800605D5286B10218843E168084358
:100D800028630020F8BD0000001002400070004001
:100D900088130000F8B5044644480E460068C007B2
:100DA000C00FB0420AD241480168490849003143A6
:100DB00001600068C007C00FB0425CD120783C4F92
:100DC000800705D57868F0218843A16808437860DA
:100DD0002078C0073FD06068012813D03968022806
:100DE00013D08907002946DA796889088900014308
:100DF0007960FFF703FF0546606801280DD00228DF
:100E000017D024E039688903ECE78901EAE7FFF7A6
:100E1000F5FE411B2748814217D878680007800FEC
:100E20000128F4D117E0FFF7E9FE411B2148814278
:100E30000BD878680007800F0228F4D10BE0FFF789
:100E4000DDFE411B1B48814201D90320F8BD7868B3
:100E50000007800FF3D115480168C907C90FB142D7
:100E60000BD9016849084900314301600068C00797
:100E7000C00FB04201D00120F8BD2078400706D550
:100E80007868072109028843E1680843786000F028
:100E90001DF87968084A0906090F515CC8400749DE
:100EA00008600020FFF7C8FE0020F8BD00200240C7
:100EB0000010024088130000B85800080C01002000
:100EC00001480068704700000C01002010B513A015
:100ED0000FC888B06C460FC414A00FC80FC4174BBE
:100EE0005A680C20114601401548042902D00829EF
:100EF00002D0144808B010BD9102090F6C46645C22
:100F0000D96A04AB0907090F595CD20303D5FFF76F
:100F1000EBF86043EEE70C486043EBE7020304059F
:100F2000060708090A0B0C0D0E0F1010010203042E
:100F300005060708090A0B0C0D0E0F1000100240E1
:100F4000001BB70000127A0000093D00042204498A
:100F50000428086902D09043086170471043FBE7FA
:100F600000E000E015480168643101601448016840
:100F7000491C016013490868401C08601249134A63
:100F8000C868401CC860904216DB0020C86010484A
:100F9000816D491C8165016D491C0165416D491CCC
:100FA00041650C49088B002806D0401E80B208839A
:100FB000782801D97820088370470000200000209D
:100FC0001800002068000020E40000201027000026
:100FD00074120020A814002010B5FFF7C3FF10BD45
:100FE000FEE770B504461E463830049D03F012FF3C
:100FF00020462A463146583003F00CFF002070BDD1
:10100000332E303000000000FEB504460078D04D8D
:10101000C00746D068680007800F012807D06868BD
:101020000007800F022809D16868C00306D5286828
:10103000800336D5606800287ED032E001216068E8
:10104000090401280AD08A00002801D005280FD001
:101050002868884328602868904301E0286808438E
:1010600028606068002810D0FFF7C8FD064608E039
:10107000286810432860F1E7FFF7C0FD801B642853
:101080006FD828688003F7D50BE0FFF7B7FD064659
:1010900004E0FFF7B3FD801B6428F1D828688003C3
:1010A000F7D420780126800700283BDA686800071B
:1010B000800F07D068680007800F022809D1686890
:1010C000C00306D42868800715D5E068012833D10D
:1010D00011E0E0680028286815D030432860FFF749
:1010E0008DFD074604E0FFF789FDC01B0228C7D825
:1010F00028688007F7D52868F82188432169C90046
:10110000084328600EE0400840002860FFF776FDA5
:10111000074604E0FFF772FDC01B0228B0D828681C
:101120008007F7D42078000724D5E0690028686A92
:1011300010D03043686200E007E1FFF75FFD07462B
:1011400004E0FFF75BFDC01B022899D8686A80079E
:10115000F7D50FE0400840006862FFF74FFD0746F3
:1011600005E09DE0FFF74AFDC01B022888D8686AA9
:101170008007F7D4207804274007002860DA002091
:101180000190E869C00008D4E969B8060143E96143
:10119000E96901400120009101906E480168C9058C
:1011A00011D40168821511430160FFF727FD0090FB
:1011B00005E0FFF723FD0099401A642870D86548C0
:1011C0000068C005F5D5A06801280AD0002801D024
:1011D000052810D0286A400840002862286AB843D1
:1011E00001E0286A30432862A068002812D0FFF787
:1011F00005FD00900AE0286A38432862F1E7FFF70E
:10120000FDFC0099411A5448814249D8286A800758
:10121000F5D50DE0FFF7F2FC009006E0FFF7EEFCDD
:101220000099411A4C4881423AD8286A8007F5D47F
:101230000198002804D0E969012000078143E96191
:101240002078C00635D5606901280CD0401D686B38
:1012500023D038436863686B400840006863FFF739
:10126000CDFC064622E0686B38436863686B304308
:101270006863FFF7C3FC064604E0FFF7BFFC801B72
:1012800002285BD8686B8007F7D5686BF821884324
:10129000A169C900084368630BE0B8436863F4E7D9
:1012A0004CE0FFF7ABFC801B022847D8686B800737
:1012B000F7D4206A002846D069680907890F0229F7
:1012C00043D001273F060228286805D0B84328608C
:1012D000FFF794FC044633E0B8432860FFF78EFC28
:1012E000064604E0FFF78AFC801B022826D82868FF
:1012F0008001F7D4E86AE16A000900010843E86266
:10130000616AA06A084369683D2212049143084358
:101310006860286838432860FFF770FC044604E0E2
:10132000FFF76CFC001B022808D828688001F7D55D
:1013300009E0FFF763FC001B022801D90320FEBD72
:1013400028688001F5D40020FEBD0120FEBD00000C
:10135000001002400070004088130000094910B5D9
:10136000401E884201D9012010BD074C6061032155
:10137000081F01F0F3FE0020A0610720206100207B
:1013800010BD0000FFFFFF0000E000E010B50021ED
:101390000F4A0846516043009B18401C1981FF28E2
:1013A000F9DD002005230B4ADB014400A418E418F2
:1013B000401CA1821028F8DB00200923DB01440037
:1013C000A418E418401CA186FF28F8DD002010BDF9
:1013D0006C0A0020F40C002010B5402802DB00202D
:1013E000C04310BD10221143C200094B4000D21867
:1013F000C01858240D23A1529B010021C3189986BF
:10140000E300C0188186034800685065084610BD97
:10141000F40C00201001002070B5104D0646014666
:101420002846FEF777FE0E4C2061FFF749FD29465E
:10143000FEF75AFEA0600B48314600680546FEF7ED
:1014400053FEE0602A46002307480F21FEF776FE90
:101450002080206964306060002070BD40420F0031
:101460001C0000200C01002000004042034610B583
:101470000020024602E09C5C6040521C8A42FADB7B
:1014800010BD0000F8B508460D460978552901D071
:10149000252903D0012A01DD451C521E344F60244A
:1014A00079792B786143334C0919334C252B30D093
:1014B000A3685B1CA360CB695B1CCB61B978002976
:1014C0000FD0F97800290FD001292C4913D0072318
:1014D0001B02C9180A7501462948FEF766FE00205E
:1014E000F8700020C043F8BD2549264B55390A75D0
:1014F0000146224807E037235B01C9180A750146F7
:10150000204B1E482033C018FEF74FFEF878401CD1
:10151000E6E76E79802E06DDE068401CE060086A30
:10152000401C0862DDE7334608339A4208D2086A55
:10153000401C0862E068401CE0600220C043F8BD27
:10154000B11DFFF793FFA919897981420DD0206958
:10155000401C206179796020414306480818416A9F
:10156000491C41620320C043F8BD0020F8BD0000C3
:101570004C0000205C05002028030020F40C002013
:1015800009140020D5060000F8B50E4604462520B3
:10159000069F079D089920706270A670E3702771FE
:1015A0002F46002008376619372B1AD009DC1A4657
:1015B000303A130003F05AF9072615152626261788
:1015C0002600612B0DD006DC382B0AD0412B08D029
:1015D000422B17D105E0622B03D0632B01D0642B83
:1015E00010D1657102E06571002D03D02A46A01D5F
:1015F000FEF7DBFDA91D2046FFF738FFB0710D2077
:10160000F0713846F8BD0000F1B584B0FFF7F6FA86
:101610000446FFF725FA524DE979002906D0297AC8
:10162000002903D0E968411A322905D8E9687D22EA
:10163000411AD200914263D9297A4A4A4A4E002976
:1016400061D06B79602701217B43F15064215164A3
:101650006979491CC9B26971EA7A914208D9A96AC3
:10166000411AE962A862A979491CA971012169712D
:101670003E49098A3E4B6A793E499F5C0F709B1830
:101680005B784B706023384E5343F3588B700026C1
:10169000CE700C71270A4F71270C8F71270ECF71F6
:1016A0006F46E8603878AF798008BF078000BF0FC9
:1016B00038436F463870002B4ED0EF2318403870F7
:1016C000009008232A480193029141230021103001
:1016D000FFF75AFF264902461031049802F0F0FB4A
:1016E000687960214843204940184168491C41609D
:1016F000C268E9688A1A4263C1606C63EE712E7237
:10170000002005B0F0BD696A491C69621A494B683E
:101710005B1C4B60697960238C4659438E4689195E
:101720000B695B1C0B614B695B1C4B61EF79002FF4
:1017300002D18F6A7F1C8F628F69BB4200D98B6197
:10174000032B85D900217346F150C8239364084BBD
:101750006246103B99547BE710231843AFE7000023
:101760004C000020741200205C050020A81400200A
:101770004C0400205C08002028030020F7B50878FE
:1017800086B00C46552801D0252802D0012A00DD5C
:101790004C1C424E62797079602104904843404964
:1017A0004518A868401CA860084680380390314658
:1017B0000B6BC968E778591A3346A0789B69303FAC
:1017C00000933B0003F052F813420B1742424229A8
:1017D000424242424242424242422C454200314948
:1017E000A3790B542179A01D32230192009102901C
:1017F0000021049A22E07161009A914200DDB161FA
:10180000284AA37913540020E9626861286B884252
:1018100000D229630120307218E00120F07115E038
:101820002048A179017010300078A0712179A01DA5
:101830000192009102904223317900220398FFF730
:10184000A3FE02460399069802F03AFB002009B075
:10185000F0BD7161009A914200DDB161114BA27936
:101860001A54114B181809239B01C018C2740F4851
:10187000008A0020E9626861286B884200D22963EF
:101880002046677A0A30FEF7B4FC617B0002000A4A
:1018900009060843B90069188863BBE74C000020BB
:1018A0005C0500203C040020F40C0020A81400205B
:1018B000F7B515460C46FFF7D3F81A4E306321787A
:1018C0000020552903D1012D01DD641C6D1E3178E6
:1018D00000290FD00127F7712A4621460098FFF70B
:1018E000D1FD002805D137722A4621460098FFF71E
:1018F00045FFFEBD71780029FBD00B4E2A46B06B28
:101900002146401CB063009800F012F80028F0D186
:1019100006482A46406C30652146009800F080F861
:10192000FEBD00004C0000205C0500207412002069
:10193000F0B508460D460978552901D0252903D070
:10194000012A01DD451C521E297800231A4FDB4372
:101950001A4C252906D0A068401CA060386C401C99
:10196000386409E014496E79896C491C802E05DDC4
:10197000E068401CE060B9641846F0BD33460833A7
:101980009A4206D2B964E068401CE0600220C0437D
:10199000F0BDB11DFFF76AFDA9198979814208D010
:1019A0002069401C2061F86C401CF8640320C0438F
:1019B000F0BD0020F0BD00005C05002028030020E1
:1019C000F8B5FFF74DF8134B1A69197900291FD0A4
:1019D0005C7A1149002C05D07D20800148640020EC
:1019E000587215E00C4E0D4C851A8036A54204D96C
:1019F0007D2292018A64012206E01219904207D9E1
:101A00007D2292018A6402228A67C8671869306061
:101A10000020F8BD4C00002074120020E02E0000D1
:101A2000F7B5087884B0552802D1012A00DD491C99
:101A30004F480268521C02604E4B4A7948784E4E1D
:101A4000039335791C468034A84208D0FF2806D07D
:101A5000606C401C60640020C04307B0F0BDA84229
:101A600001D0FF2875D1306B009030610120707279
:101A70004048CF7890380078372F76D007DC303F59
:101A80003B0002F0F3FE0672137272722172612F34
:101A90006BD004DC382F68D0412F66D11DE0622F57
:101AA00063D0632F61D0642F5FD153E0314B8F79C6
:101AB000A03B1F70887100983061881D097932231E
:101AC00001920091029037E00020097936230091BD
:101AD000019002460290012130E0264B8F79A03B15
:101AE0001F70CF7A8B7A3F02DB19F361B37A88716A
:101AF00098004B720019078F8F72078F5B1C3F0A8B
:101B0000CF72876B3F0C0F73806B000E4873D8B297
:101B1000B0720A2801D30020B07208796B461870A1
:101B2000C00603D57D20154B80019864881D097976
:101B30004223019200910290002229460398FFF768
:101B400023FD0246E06B401CE0630399049802F019
:101B5000B7F90AE0CA798879120280180A7A497AB4
:101B60001204090651184018F061002075E70000C2
:101B700028030020DC0400204C0000207412002008
:101B8000034610B50020024602E09C5C6040521CF7
:101B90008A42FADB10BD30B50D4608460978144676
:101BA000252901D0012030BD062C01D2032030BDF3
:101BB000611EFFF7E5FF29192039C97F814201D055
:101BC000042030BD002030BDF8B51E460B46552719
:101BD000069D0799077043708270C67004460571B0
:101BE0002A46401DFEF7E1FA691D2046FFF7C8FFAF
:101BF000014660194171A81D052E02DA002E00D1A0
:101C00000020F8BDFEB516460F460546FFF7C3FF98
:101C1000040014D0684604720420009002A90B4806
:101C200001910278401E0178EE230948FFF7CCFFAE
:101C300002460749284602F043F92046FEBD3246D7
:101C40003946284600F006F8FEBD00008500002059
:101C5000EC080020F7B5FA4886B04F7842688260F9
:101C6000421C15788E782D0936072D01360F0B7919
:101C700035431570F34A029200780C46049087426F
:101C800001D0FF2F77D12146E6780931EE488C4606
:101C9000332E72D028DCED49182E0A686CD012DC85
:101CA000072E20D008DC002E65D0012E3ED0032E5A
:101CB00041D0052E7ED160E0112E7CD0162E7BD037
:101CC000172EF7D13FE2232EEED006DC192E74D06A
:101CD000212E73D0222EEDD18FE1242EE4D0312E8F
:101CE0004BD0322EE6D1BFE0582E68D012DC542EF5
:101CF00066D008DC342E71D04F2E70D0502E6FD0AD
:101D0000532ED7D16EE2552E6BD0562E6AD0572E59
:101D1000D0D164E2304663380421030002F0A6FD0E
:101D200009F0EFEE171D4A104A154A00641D009392
:101D30000194012351E2C649182003E03946C7E265
:101D4000C4490C200191009005E0C348F6E1C24966
:101D500010395020F6E733463FE2E1790020B94AD6
:101D600003E023185B7A1354401C8842F9DBB54822
:101D700002F0DEFCA3E075E2EEE1A27961791202E5
:101D80008918E27989B2882B2DD0892B2FD08A2B04
:101D900031D0832B34D0842B37D0852B3AD0862B6F
:101DA0003DD0872B40D08B2B43D08C2B46D0FE2BA5
:101DB0001DD006E097E29FE1AEE1EDE1C9E066E209
:101DC00027E2A92B3FD0B32B41D0992B42D0A12B96
:101DD00045D09C481038401800925FE244E0F6E19C
:101DE000F1E140E249E2490009189C483AE0490023
:101DF00009189B4836E0490009189848203831E016
:101E000049000918952080002CE0490009189D2000
:101E1000800027E049000918A520800022E0490041
:101E20000918FD2080001DE0490009188B48A038E2
:101E300018E049000918DD20800013E04900091866
:101E4000BD2080000EE04900091886480AE04900DC
:101E5000854807E0854849000818001DBCE749008F
:101E60000120C0060818B7E7A27961791202891823
:101E7000E27989B2882B25D0892B27D08A2B29D0CB
:101E8000832B2CD0842B2FD0852B32D0862B38D08F
:101E9000872B3BD08B2B3ED08C2B41D0FE2B45D0BB
:101EA000A92B47D0B32B49D0992B4AD0A12B4BD08B
:101EB00064481038401800226146FEF776F9002089
:101EC000009024E149000918644840E049000918DD
:101ED00063483CE0490009186048203837E0490071
:101EE00009189520800032E0490009189D208000E3
:101EF0002DE049000918A520800028E0DFE1D2E1AB
:101F0000CEE149000918FD20800020E049000918B1
:101F10005248A0381BE049000918DD20800003E08A
:101F200049000918BD2080000818C4E749000918B5
:101F30004B48F9E7490009184A48F5E749004A487B
:101F4000F2E74900494802E049000120C0060818AC
:101F5000B2E7A2796179120289180922920189B245
:101F6000002B0FD0012B13D0022B1CD0032B20D021
:101F7000042B26D0052B2AD0062B28D0082B34D0B2
:101F800000202AE00B095B00181833E0012024E050
:101F90000B095B00181811E00A07120F012191408C
:101FA0000840F3D119E00A09520010180522D201A5
:101FB00020E00A09520010180F2292018018808E2A
:101FC000EAE70A09520010180122920212E0C90041
:101FD00008184030007E4006C00F69460873012093
:101FE00003A9212301910090F7E00A09520010187B
:101FF0000922D2018018808ACEE7A2796179120283
:10200000891889B2002B33D0012B3AD0022B41D052
:10201000032B48D0042B4FD04022052B54D0062B45
:1020200052D0072B5BD00020694608730020009037
:10203000034803A9401C0191027822237EE6000098
:1020400084000020EC080020F40C00206C0A002022
:10205000EA570008ACF7FF1F107C0008B40400002A
:10206000B4050000B40600005C050020740C0020DC
:102070000B070909490009181B0F9520E279800018
:1020800035E00B070909490009181B0F9D20E2796B
:1020900080002CE00B070909490009181B0FA52037
:1020A000E279800023E00B070909490009181B0F9A
:1020B000FD20E27980001AE00B0709091B0F490097
:1020C0000918E2798D4812E0C90008184030018BE8
:1020D0009143E279D207520E11430183A6E70B0721
:1020E0000909490009188548E2791B0F8030081852
:1020F000194601F009FF99E7002B05D0012B00D00C
:10210000DDE602F0B7F8DAE602F0ECF8D7E6019087
:102110007B48E378027811E6A179607909024018DA
:10212000E179784A80B2002B0AD0774C012B03D09A
:10213000764B9B8A002B03D0400000190091ADE044
:1021400040008018FAE7002A01D000200860002033
:1021500000901723019040E0002A01D00020086081
:10216000A17960790902401885B2E27900206849B6
:1021700003E02618767A0E54401C9042F9DB64493D
:10218000284602F0E3FA00200934009001905C48F0
:10219000039402781823D1E5A179607909024118E6
:1021A0005A48C182818A00290BD000218182574878
:1021B00001F010FE00200090019051481923027890
:1021C000BCE50121F2E751480383002002E04F49BA
:1021D0000020088300900190E3782A46AEE54B4941
:1021E0002020AFE5A179607909024018494980B201
:1021F0000A18E179121D782801D3002105E00B1897
:10220000782B02D97821081A81B2C8B201920090C5
:10221000A1E5A1796079090240183E4980B20B1806
:10222000E2791B1D782801D3002205E011187829D6
:1022300002D97821081A82B261461846FDF7B5FF27
:102240000020009001902E48E378027839460298E9
:10225000FFF7BAFC02460299069801F031FE2D48BC
:1022600002F094FA3CE02B4802F090FA0020009033
:10227000019023485523027860E5244801F0AAFD27
:102280000020009001901E485623027856E5032155
:1022900009022148FDF7A2FF0020009001905AE5B5
:1022A0001E481F4A4DE7A179607909024018E1797B
:1022B00080B20D01FEF756FBE9B2009127E7FEF769
:1022C000E9F80020009001900D486523027835E57B
:1022D0000298FFF779FC02460299069801F0F0FD9A
:1022E000002009B0F0BD02206946087303A901204F
:1022F0000191EE232A4600900499E9E714040000B6
:10230000850000200080000800A00008A81400201C
:10231000EC080020740C00205C050020F40C002068
:10232000F405000070B5FEF77FF8164800F070FA6B
:10233000154D164C6869A0651248816861658188F1
:10234000491C81808088E0640E4801F043FD2868C4
:10235000206768686067A868A06701220C4B114677
:10236000A06DFDF7F5FF20468030E9680160A9699E
:102370004160E96981602969C160296A01610020C1
:1023800070BD0000A81400209800002074120020E6
:102390003930000008B504494A6902434A61496975
:1023A0000140009108BD00000010024008B504493A
:1023B000CA690243CA61C9690140009108BD0000B1
:1023C0000010024008B504498A6902438A6189699C
:1023D0000140009108BD00000010024070B5094E98
:1023E00004467618203E049D0C34F17F0830102DF1
:1023F00003D00A50F07F035170BD0A51F17F0B509A
:1024000070BD0000C4530008044A51182039C97F28
:10241000425852085200425070470000C45300080E
:10242000044A51182039C97F425801231A434250A7
:1024300070470000C4530008044A51182039C97F6E
:10244000425802231A43425070470000C453000808
:10245000054B10B559182039C97F4358032424036C
:10246000A3431343435010BD94580008054B59181B
:102470002039C97F001D0B581B0C1B0413430B5044
:1024800070470000C4530008054B10B55918203997
:10249000C97F4358034C23401343435010BD0000F1
:1024A00094580008EFBFFFFF054B10B559182039AD
:1024B000C97F43588024A3431343435010BD0000F9
:1024C00094580008054B10B559182039C97F435856
:1024D0000324A402A3431343435010BD945800089F
:1024E000054B10B559182039C97F43582024A34300
:1024F0001343435010BD000094580008054B10B51D
:1025000059182039C97F43584024A34313434350EB
:1025100010BD000094580008054B10B5591820391B
:10252000C97F435803242402A3431343435010BDDF
:1025300094580008F0B500233CE001249C40224060
:1025400037D04F6806681446544365006519AE439A
:1025500067433E4306604E68012E01D0022E05D12E
:102560008F6886686743AE433E4386600F69C668DE
:10257000AE4325467D432E43C6604D68022D18D1DB
:102580004D69FF2A09D8066A544354432201121B9D
:1025900096436C43264306620BE0140A22466243CC
:1025A000624362431401A61A446A6A43B443144363
:1025B00044625B1C0A681446DC40BED14A68012AAA
:1025C00001D0022A06D10A68C968436893434A4386
:1025D000134343600120F0BD0069814301D0002016
:1025E00070470120704710B5044601F0BDFA206025
:1025F00001F0A0FA606001F0ABFAA06010BD00002D
:10260000014610B5002000290FD1104A116B89072F
:10261000890F01290AD0022911D0032909D001F01C
:10262000A3FA01F087FA01F093FA10BD01F09CFAC9
:1026300010BD11688907C90FFAD0054810BD116A8D
:102640008907C90FFAD00120C00310BD0010024055
:1026500000127A0010B5036800225B06DB0F25D15B
:102660000CC98C681A434B6823431A43CB681A433E
:102670000B691A434B691A438B691A4303680C4C64
:1026800023401A43026042680A4B1A40CB681B0C75
:102690001A430B681A43426001238A695B030839B5
:1026A0009A4202D1898C89B201610122104610BD83
:1026B0004000FFFFFBF0FFFFF0B50268194B1A4C1A
:1026C000984201D0A04203D17025AA434D682A4305
:1026D000164D174E174F98420AD0A04208D0164CFC
:1026E000A04205D0A84203D0B04201D0B84204D1E4
:1026F00003242402A243CC68224302608A68C26297
:102700000A888262984205D0A84203D0B04201D024
:10271000B84201D1097C0163416901221143416141
:102720001046F0BD002C0140000400400040014074
:10273000004401400048014000200040416801225F
:10274000D2029143416081680822914381607047C1
:10275000FEB5044600680D460026C007C00F43D1F1
:10276000E9686868AA690843296911430843216830
:102770001E4A114008432060A868616803221203C2
:102780009143014361606869A1681211914301435B
:10279000A1601748844203D10020FFF731FF06E013
:1027A0001448844220D16846FFF71DFF0298002894
:1027B0001AD02968002917D00126AA69F3039A4282
:1027C0000CD140004A088018FDF78EFC0A4980B2FF
:1027D00001400007420F0A43E26005E04A08101872
:1027E000FDF782FC80B2E0603046FEBDF369FFFF7A
:1027F0000038014000440040F0FF000010B5802286
:102800000249FDF7D2FC002010BD0000045800086A
:10281000F0B5154A00215514144C154F0CE0D65A4A
:10282000BE4208D19B185B886668B34203D90AC4CC
:102830004B1C2360083C491C4B01AB42EFD3216881
:102840000123002905DB49018918202201F0C2F982
:1028500000E08380A06840012030A84201D9002018
:10286000A0600020F0BD000000C800089800002013
:10287000AA5500001FB50B46024604A1684601F0A8
:10288000E1FF0146684601F033F91FBD201B5B25BF
:10289000643B25644800000010B50120FFF77AFD75
:1028A00000210A2000F038FC0A2000F02BFC002157
:1028B0000B2000F031FC0B2000F024FC10BD0000C8
:1028C000F0B5012087B04004FFF764FD01208004CB
:1028D000FFF760FD0120C004FFF75CFD01208005CB
:1028E000FFF758FD0126C020002403256A46049600
:1028F00031C20927FF0669463846FFF71BFE8020D4
:10290000694631C1694638460494FFF713FE9320A7
:10291000000100900394694601960295049438469C
:10292000FFF708FE3002B86168026A46049631C2B9
:1029300069463846FFF7FEFD29486A46049631C2CB
:1029400069462848FFF7F6FD27480090039469463A
:102950000196029504942348FFF7ECFD07204003FD
:102960000090029403946946019604941F48FFF76F
:10297000E1FDF0206A46049631C269463846FFF709
:10298000D9FD3002B86140006A46049631C26946FA
:102990001448FFF7CFFD40206A46049631C26946CD
:1029A0001348FFF7C7FDF0020090694601960295B3
:1029B00004943846FFF7BEFD8020009069460196DA
:1029C000029504940A48FFF7B5FD40206A46049634
:1029D00031C269460348FFF7ADFD07B0F0BD000006
:1029E0000704000000040048C0FC00000008004884
:1029F00000140048084807490160084901600421A3
:102A00004160074A8260C1684907FCD102610549FB
:102A100001607047CCCC00000030004055550000EC
:102A2000FF0F0000AAAA0000F0B591B0282106A867
:102A3000FDF7D4FB18216846FDF7D0FB0120000309
:102A4000FFF7C0FC01208004FFF7A4FC0024082548
:102A500002260327039404946A460594E0C269465B
:102A60002248FFF767FD102069460394C1C1012089
:102A70000490694605941D48FFF75CFD20200394EF
:102A800004946A460594C1C269461848FFF752FD8E
:102A90000021192000F040FB192000F033FB072033
:102AA00000020890012006940A9040020B900994BD
:102AB000802007940E940D9007200D4C0F900C95DC
:102AC00006A92046FFF7C6FD6068102188436060B4
:102AD0006068A843606060680902884308436060DA
:102AE000206840210843206011B0F0BD0004004878
:102AF0000030014010B586B014216846FDF76EFB2A
:102B00001020FFF753FC0021112000F005FB1120DD
:102B100000F0F8FA2F20694608800020019008484C
:102B2000084C02902046FFF7C7FD206880218843AB
:102B30002060E06801210843E06006B010BD00009D
:102B4000E70300000010004070B501208EB0800344
:102B5000FFF738FC03204002079002200890032072
:102B600000240990012509200A9407A90C950B94CB
:102B7000C006FFF7DFFC3A4E102202213046FFF775
:102B800083FC002202213046FFF762FC0022022172
:102B90003046FFF7A5FC002202213046FFF7AEFCCD
:102BA000802202213046FFF77FFC002202213046BE
:102BB000FFF7B2FC002202213046FFF783FC00221F
:102BC00003213046FFF760FC002203213046FFF767
:102BD0003FFC002203213046FFF782FC0022032144
:102BE0003046FFF78BFC802203213046FFF75CFC68
:102BF000002203213046FFF78FFC002203213046DC
:102C0000FFF760FC00211B2000F086FA1B2000F07B
:102C100079FA14486946006800900194029403947C
:102C2000059406940C20104C04902046FFF790FD6C
:102C30006068290508436060606849000322520506
:102C4000904308436060A06849120843A060204692
:102C5000FFF774FD2068284320600EB070BD0000AF
:102C600000000240340000200038014070B58EB0F2
:102C70001C216846FDF7B2FA182107A8FDF7AEFA45
:102C8000012464042046FFF791FB2046FFF782FBF6
:102C90000E200790022008900320012509900024AF
:102CA00009200A9507A90C950B94C006FFF742FC72
:102CB000414E102204213046FFF7E6FB002204219A
:102CC0003046FFF7C5FB002204213046FFF708FC21
:102CD000002204213046FFF711FC802204213046F7
:102CE000FFF7E2FB002204213046FFF715FC00222B
:102CF00004213046FFF7E6FB002205213046FFF7AE
:102D0000C3FB002205213046FFF7A2FB002205216C
:102D10003046FFF7E5FB002205213046FFF7EEFBCA
:102D2000802205213046FFF7BFFB002205213046F7
:102D3000FFF7F2FB002205213046FFF7C3FB00211D
:102D40001C2000F0E9F91C2000F0DCF9A61EFF2190
:102D5000304600F0E1F9304600F0D4F91748EE03B0
:102D6000006800900194029403940C2004AA51C2BC
:102D7000134C69462046FFF7EBFCA068211408437A
:102D8000A060A068B0433043A06020681F214905BF
:102D90008843084320602068491188430843206025
:102DA000A068A1140843A0602046FFF7C7FC206874
:102DB000284320600EB070BD0000024038000020A3
:102DC0000044004000B50846042A02D80020C04351
:102DD00000BD01787F2902D90120C04300BD4178A0
:102DE0004906490E1F2902D90220C04300BD1146E1
:102DF00001F0DAFF0028F9D0042000BDF7B588B053
:102E00000F460A9A0898FFF7DDFF0690002803D0C6
:102E10000020C0430BB0F0BDB6483A780078394680
:102E200082427DD18C784A78CB78B98824024DBA19
:102E3000B1491C4308704A70012007902005210702
:102E40000226000E090F130001F010FD119E0A4723
:102E5000859FB7D59E9E9E9E9E9E9E9EE1F39E0060
:102E6000E81DC008A4490390887000202FE00020CE
:102E700000900120019002980027C00004901CE0FF
:102E80002005000E42009D482107121809208001EC
:102E90001018090F808EFDF7DBFC002803D0019984
:102EA0000098084300900198641C4006000E7F1CA7
:102EB000A4B20190082F03DA0498C019A842DFDBFE
:102EC0008D49029A00988918C8700298401C03998D
:102ED00002908842CBDB761855E0E81DC008864991
:102EE00003908870002031E00020009001200190C4
:102EF00002980027C00004901EE02005000E42004A
:102F00007E4821071218092080011018090F808AB5
:102F1000FDF79EFC002805D001990098084300E0C9
:102F2000E5E000900198641C4006000E7F1CA4B2EE
:102F30000190082F03DA0498C019A842DDDB6E491E
:102F4000029A00988918C8700298401C0399029050
:102F50008842C9DBBFE76800674984468870002063
:102F60000EE021184A006549470052180921C9019D
:102F70005118898E604A0B0ABA18D3701171401C1F
:102F8000A842EEDB17E0761C87E068005A4A8446C8
:102F9000907000200DE021184B00584947005B1845
:102FA000092189015918898ABF180B0AFB703971E8
:102FB000401CA842EFDB6644E5E7002D12D0FF225B
:102FC0001202954207D142004C4812189D20800001
:102FD000101800F091FF394647480A9AFDF7E5F8C6
:102FE0000A9E7FE04200454812189D20800010187C
:102FF00000F042FEEFE738797979000208433F4953
:10300000620052180921C90151188886E3E7E81DBA
:10301000C008394903908870002030E03818C07922
:10302000009001200190002005900298C0000490BB
:103030001FE036E02005000E42003048210712183C
:103040009D20090F80001018009B019A1A4202D09F
:1030500000F052FF01E000F00FFE0198641C4006F2
:10306000000E01900598A4B2401C0590082804DACF
:10307000049805994018A842DCDB0298401C03998B
:1030800002908842CADB1C48B9788170F978C17017
:103090003979017179794171361D0698002814D06B
:1030A00025E000200EE04100C919CA79097A120210
:1030B0000A4321184B0011495B180921C90159180D
:1030C0008A86401CA842EEDBDDE70798002809D07D
:1030D000B1B2094801F068FE07498855000A89190C
:1030E0004870B61C32460449089800F0E9FE0020FA
:1030F00090E6000090000020EC090020F40C002075
:1031000070470000C106C90E0120884001490860CF
:103110007047000000E100E08307FF22DB0E9A40C9
:103120008907090E994000280BDA0007000F0838BC
:10313000830808489B001818C36993430B43C36175
:103140007047830804489B001818036893430B4397
:103150000360704700ED00E000E400E08307FF2219
:10316000DB0E9A408907090E994000280BDA000708
:10317000000F0838830808489B001818C369934358
:103180000B43C3617047830804489B001818036809
:1031900093430B430360704700ED00E000E400E060
:1031A000F3B5074681B0002000903D78FF206E0700
:1031B000EC08760FE40001F039FE802C01D20020EB
:1031C000FEBD324601265C495C48130001F04EFB0F
:1031D0000805313539898D91A1B057490978002901
:1031E00003D0554949788C4220D18188544F491CDD
:1031F00081803D70504D3021A87808437870E87880
:103200000843B8703520F87004213846FDF7FCF803
:103210003021084338710D207871112001F006FE2D
:103220000621384600F016FE6C702E70424806717A
:1032300062E0C188491CC1805EE00189491C0181AE
:103240005AE00A78002A02D04A78A24201D00E71D0
:1032500052E042893849521C42810020CA780EE06F
:103260004100C9194B7889781B010907090F5B18C0
:1032700034490C181321490161180B75401C2E4C60
:103280009042EDDB2E4A002015702E4F0FE00921F1
:103290003B1889015B18197D0D09410089183035EB
:1032A0004D701B7D1B071B0F30338B70401CA178AA
:1032B0008842ECDB0806C00D401CC1B22048FDF777
:1032C000A3F830210843A1781D4A49008A1850709C
:1032D0000D209070C91CC9B2194800F0BBFD2671C1
:1032E0000AE08189491C818106E0C189491CC181AC
:1032F00002E0018A491C018202980007C10E1148B0
:103300000918132080010818818C491C81840098B9
:10331000FEBD428A521C42820878002897D0487825
:10332000A04294D10120C0020922D20690618EE70A
:10333000028B521C02838AE7C8000020B4110020CF
:10334000C8140020F40C002010B501200449C00668
:10335000486004480168491C016000F005F810BD90
:1033600000ED00E03000002070B50E480178002428
:10337000002905D004700C4801780C48FFF710FFB5
:103380000B4DE86F00280BD00A4E0B490220326823
:10339000FEF78EFA3460EC678021074801F040F9AF
:1033A00070BD0000E0000020E100002008150020B2
:1033B000A802002040000020BC03002010B50648F1
:1033C000054B00780021403B5A1840325478491C84
:1033D00014700F29F8DB10BD340D002010B5084C17
:1033E000084B01220221A06DFCF7B2FF064800F055
:1033F000F1FCE06D401CE065A06D2066002010BD72
:103400007412002039300000A81400200248C16D59
:10341000491CC1650020704774120020F3B5FA4DB5
:1034200085B0286800286FD0686800281CD000226A
:103430000D21082000F080FD00221146082000F038
:103440007BFD01221146082000F076FD0020014698
:10345000EE4A13184033401C19701028F8DB002680
:103460000121144640347BE20122E1E7B2000598D5
:10347000059B805CD7187A78019201257B880093A0
:103480001B2873D012DC0246030001F0EFF91B5C2D
:103490007272727272723E3E3E3E3E3E5C5C5CA751
:1034A000A7A73E3EBEBEBEBEBEBE5C00342870D0E6
:1034B00011DC01461C390B0001F0D8F918A7A7A7A9
:1034C000A7A7A7A7A7A7A7A745454545454545459C
:1034D00045454545F7453A2873D008DC014635395E
:1034E0000B0001F0C3F905E26E56E26E3000DC28F5
:1034F00004D004DC3B28EFD0C82824D120E1DD280B
:10350000FCD0FA28F9D11BE133E2D01F030001F00F
:10351000ADF90E080A10181B1D1A1A1A1A1A1A20C9
:10352000261A207C4AE0FFF749FF00281FD0207CA4
:103530003AE0FFF743FF002816D1207C002813D182
:1035400025E000F0C3FAF5E12078F7E7FFF736FF52
:103550001DE0207C00280AD0002905D007E0207C4F
:10356000002804D1002902D0012010E04DE0002005
:103570000DE0130001F07AF9070C050E111B262E41
:103580000C0000F0A3FA00990198FDF775F920747A
:10359000D0E11AE100F09AFA0CE0207C0028E6D095
:1035A00000990198FDF768F90028E0D0DCE7207C5D
:1035B0000028DCD000990198FDF75EF90028D6D1EB
:1035C000D2E758E1207C0028CED100990198FDF780
:1035D00053F9B3E7207C0028ECD0C5E7102804D0CD
:1035E000112804D0122AAED10AE0227C03E0207C0C
:1035F0000028A8D001220099019800F09DFC99E1D3
:10360000207C00289FD00022F5E715383D79030083
:1036100001F02CF9120A1215181B0F1E3C4C5B6AA4
:103620002D798185898D7D9400F050FA13E0207406
:1036300084E000F04BFA1DE000F048FA29E000F0C9
:1036400045FA36E000F042FA42E000F03FFA4EE080
:10365000207C002870D028460099FDF795F9054692
:10366000F9887879FDF790F9854263D064E0207C91
:10367000002861D028460099FDF786F90546F988AB
:103680007879FDF781F9854254D155E0207C0028F6
:1036900052D028460099FDF777F90546F9887879E0
:1036A000FDF772F9854245DB46E0B1E0207C002859
:1036B00042D028460099FDF767F90546F9887879E0
:1036C000FDF762F9854235DC36E0207C002833D0F6
:1036D00028460099FDF758F90546F9887879FDF7ED
:1036E00053F9854226DD27E0207C002824D0284697
:1036F0000099FDF749F90546F9887879FDF744F90D
:10370000854217DA18E0207C002813D1A3E7207C3B
:1037100000280FD1AEE7207C00280BD1B9E7207C30
:10372000002807D1C5E7207C002803D1D0E7207C02
:103730000028DCD001207AE7002078E70225F9E0B4
:103740003F791546C8280DD0DC2823D0DD282AD0A3
:10375000FA28F3D12D48E90008184030007EC00651
:103760002AD508E02948E90008184030007EC00644
:1037700001D4002121E0207C002822D03846009985
:10378000FDF702F90146284600F07EFA284600F0CF
:10379000F5F84CE71D48E90008184030007EC006E7
:1037A000E9D4012109E01948E90008184030007EF9
:1037B000C006E0D4022100E003212846FDF70CFEFC
:1037C000D9E7284600F0AEFDE0E73F79022534282E
:1037D00002D0372816D108E0207C002812D03846C5
:1037E0000099FDF7D1F8401C07E0207C002809D0A3
:1037F00038460099FDF7C8F8401E02463846009941
:1038000000F012FC96E000006C0A0020F40C00208E
:103810003D7979790291F9880191332814D03528BE
:103820001BD038288AD1207C002887D00298FDF749
:10383000ABF8074628460099FDF7A6F83A1A019911
:10384000029800F0F1FB79E7207C0028FBD02846A5
:103850000099FDF799F80246F1E7207C0028F2D0A4
:1038600028460099FDF790F8054601990298FDF762
:103870008BF82A18E3E73A7979790291F98801916E
:10388000797A03917D89362806D0392812D03A28D2
:103890001FD03B284DD131E0207C002849D0104674
:1038A0000099FDF771F8074601990298FDF76CF849
:1038B0003A180CE0207C00283BD010460099FDF718
:1038C00063F8074601990298FDF75EF83A1A29460F
:1038D0002CE0207C00282CD010460099FDF754F8ED
:1038E00007B201990298FDF74FF800B247433A46F4
:1038F0002946039800F098FB3A1416E0207C002833
:1039000017D010460099FDF73FF807B201990298C9
:10391000FDF73AF801B23846FCF7FCFB02B20F465D
:103920002946039800F080FB3A46691C039800F092
:103930007BFB0325301141000F4801230818310794
:10394000090F02898B401946114000D00121277CC4
:103950000830002F01D01A4300E09A430280761904
:103960000698864200DA81E503494868401C4860B1
:10397000002007B0F0BD00006C0A0020FEB507462D
:10398000402802DB0020C043FEBD2C48F9000E1881
:1039900000964036348BE10601D40020FEBDA1061E
:1039A0003CD561063FD42649096800980A25406D38
:1039B0000190081AA1070FD0A107890F012905D08E
:1039C000022905D0E143890705D005E0642503E01D
:1039D0007D25ED0000E01B4DA84224DB2946FCF7C5
:1039E00099FB014615487A0012180B208001101827
:1039F0008446808E019B401869435B18009980B211
:103A00004B650D2189015118898E814203D80846E2
:103A100040210C4334836146888604E0600602D569
:103A2000402084433483307EB9B24006C20F052063
:103A300000F082FA307E4006C00FFEBDF40C00207C
:103A40001001002010270000F7B50446FCF777FFAF
:103A5000054602992068A942A16806DC4018029A2E
:103A60000199FCF7A2FB029919E040182A46019936
:103A7000FCF79BFB29462046FCF7B0FC2046FCF7F0
:103A80005EFF06460298471BB7420DDCA16820681E
:103A90003A46401801994919FCF787FB39462046F8
:103AA000FCF79CFC0298FEBD002E0CDDA16820688E
:103AB0003246401801994919FCF777FB31462046F8
:103AC000FCF78CFCAD192846FEBD0000074A0F200C
:103AD00011183F235B5C4031401E0B700028F7DC5F
:103AE00002494031087C087070470000F40C002047
:103AF00010B50C460A4601460348FFF7A5FF00F043
:103B000077FD204610BD00006C02002010B50C4669
:103B10000A4601460348FFF797FF00F069FD20467B
:103B200010BD00006C02002010B50C4600F0C8FD6E
:103B3000204610BD04494968F0221140034A090992
:103B4000515CC8407047000000100240B85800089F
:103B500003494968034A4905490F515CC840704709
:103B600000100240C858000810B5074841680C20F2
:103B70000140064805D0042904D0082901D100F0ED
:103B800009F810BD024810BD0010024000127A0072
:103B9000001BB70010B50C4C6168012212040B48E1
:103BA000114002D0914200D10948E16A0907090F8A
:103BB000491CFCF799FA61680F2292041140890CA4
:103BC000891C484310BD00000010024000093D0060
:103BD000001BB70070B5D417A40F0023A418A510BC
:103BE00003E09C000E5906515B1C9D42F9DCD40F8A
:103BF0006B00A418651003E05C000E5B06535B1CB1
:103C00009D42F9DC104670BD0920C006006901091B
:103C10000F20884370470000F8B5002384468025B4
:103C2000DB431248002421462A464A4312181788CB
:103C30000F4EB74209D17E26B75A0E4EB74204D175
:103C40005288A24201DD0B461446491C0829EBDBD1
:103C5000082B06D26B43191880226046FFF7BAFF83
:103C600002E06046FEF7CAFD0020F8BD00C0000873
:103C7000AA550000A55A00000B0702881B0F01215E
:103C800099408A430280704730B5402802DB00200B
:103C9000C04330BD0D4CC20013191A464032157E88
:103CA000AD0611D4400000190D24A4010419A18609
:103CB0000B240021A401001981860548006858657D
:103CC000108B202108431083002030BDF40C00200D
:103CD0001001002010B500F001F810BDF0B52D4F17
:103CE000B868C007C00F4DD0F8682C4DC4B22A4840
:103CF000C16A491CC162018D491C018528780028D0
:103D000002D1204601F092F828780026002819D127
:103D10002448234902788C540178491C01700D2CE9
:103D200010D10446007801F081F820781E4908700F
:103D30001E490120087026701D48067001201D498B
:103D400000074860287800281CD01B490878401CD0
:103D500008701A48026B521C02630878184A1278DD
:103D6000904210D30120C0020921C90688612E703B
:103D70001449012008700E4908700A48067012495B
:103D800080208862F0BD11480978405C387301F0EA
:103D90004DF8F0BD0030014074140020D000002028
:103DA00008150020CD000020E1000020E0000020E8
:103DB000CC00002000ED00E0CF00002074130020B4
:103DC000CE000020E200002000140048E81400208B
:103DD0007047000070B51A4C6168491C6160194950
:103DE0000180A18841801849CA6C8280496D816038
:103DF000112181831549C183A1684A0114495118D1
:103E000000250B462A469E5CFF2E04D1521C202A18
:103E1000F9D3002D10D02022FCF7D0FBA068206041
:103E2000401CA0604001012189022030884201D954
:103E30000020A060002070BD202200F0DDFCEDE736
:103E400098000020AA55000074120020A55A000016
:103E500000C8000870B503460E460807C10E134897
:103E6000002509180520C0010818818A104C491C3A
:103E70008182207A002817D1324619460D48FCF776
:103E800094F9A6710020E0710A48E179405C0A4982
:103E900008730121217200F0C9FF08498020886160
:103EA00000010921C9068862284670BDF40C002073
:103EB000C8000020E8140020003001400014004831
:103EC00010B514460A46012802D0022806D00DE09B
:103ED00021461046FFF71AFE054804E02146104629
:103EE000FFF722FE0348816F491C8167204610BD01
:103EF00014020020A80200200B0702881B0F0121DA
:103F000099400A43028070470907090F01238B403B
:103F10000188002A01D0194300E0994301807047CD
:103F20000907090F01238B400188002A01D019439A
:103F300000E099430180704770B50B051B0E204CC3
:103F40005B000D071C192D0F030000F08FFC090604
:103F50000B14191E22272C313600FF292DD895204D
:103F6000800003E0FF2928D89D20800020182946E2
:103F7000FFF7D6FF21E0FF291FD8A5208000F5E735
:103F800080291AD2FD208000F0E7802915D20D4843
:103F9000ECE7402911D2AD208000E7E740290CD2A0
:103FA000B5208000E2E7802907D206482030DDE70F
:103FB000802902D203488030D8E7002070BD00007D
:103FC000F40C0020140400000121C903034A002856
:103FD00001D091627047916170470000000800486D
:103FE00001218903034A002801D091627047916141
:103FF00070470000000800480121C903034A002857
:1040000001D091617047916270470000000800483C
:1040100001214903034A002801D091627047916150
:104020007047000000080048F0B5304C4B001C19E8
:104030000923DB01E6180B23DB01E51892B28A287D
:104040003DD00EDC294F4B00DF1909239B01FF18DF
:104050008338030000F00AFC0714181C21262D46A3
:10406000480099283ED006DC8B282CD08C2831D0F3
:104070008D2839D133E0A12834D0FE2834D131E065
:10408000102931DABA822FE010292DDABA862BE016
:10409000102929DA0520C00108E0082924DA0F20B8
:1040A000800114E008291FDA012080022018828292
:1040B0001AE0802918DAB28616E0AA8614E0802970
:1040C00012DAB28210E040290EDA0D2080012018A9
:1040D000828609E0402907DA0B208001F7E74029B2
:1040E00002DAE8E78029E8DB0020F0BDF40C0020CC
:1040F000F0B58DB0002500F015FEFCF7B1FC059081
:1041000010213A4800F070FE0790FCF7A9FC0490DB
:104110001021364800F012FE0690FCF7A1FC039037
:104120001021324800F028FE0190FCF799FC064669
:1041300010212E4800F038FE0090FCF791FC2C4A2C
:1041400004469068012108439060881E1061294848
:104150001061264B0021585C1070491C1029FADBB5
:104160001768FCF77DFC0B9001990098029701906D
:10417000214F0091781921A1069B079A00F062FB5C
:1041800045190B98A11B001B01910290039A0499F9
:104190000398B21A431A009208460599421A7819F0
:1041A00020A100F04FFB441908A8FEF71CFA26488E
:1041B00042680120000402403819134623A100F090
:1041C00041FB0419381926A1089A00F03BFB01199C
:1041D0003846FFF78DFC01210D20FEF74BFB2449EB
:1041E0000320886000200DB0F0BD0000B45300082B
:1041F0000030024001A00000140100200D0A4352CB
:1042000043202025303458202025303458202025C4
:104210003034582020253034582020253034580D93
:104220000A00000074696D65202530346420202563
:10423000303464202025303464202025303464203C
:1042400020253034640D0A00001002404D61696E73
:10425000536F75726365202578202564200D0A0050
:10426000737973636C6B202564200D0A00000000D5
:104270000000002030B50021174D0846696042005B
:104280005219401C1181FF28F9DD00200522134C32
:10429000D20143001B199B18401C99821028F8DB9F
:1042A00000200922D20143001B199B18401C99864B
:1042B000FF28F8DD00201022C100091940310B8BC6
:1042C000401C93430B834028F6DB012004492860FF
:1042D0004882002030BD00006C0A0020F40C002051
:1042E000A814002010B500210C48092201600C4BD5
:1042F000084692014400E418A418401CA186102826
:10430000F8DB0020012292024400E418A418401CAB
:10431000A1820828F8DB002010BD00006C0A0020F4
:10432000F40C002010B5402802DB0020C04310BD73
:104330000B4BC100CA18114640310C7EA4060DD5A6
:104340004000C0180B2300249B01C0188486054838
:1043500000685065088B202290430883002010BD20
:10436000F40C00201001002010B5FCF74DFCFCF708
:1043700033FE10BD70B594B030216846FBF72EFFB8
:104380000024022501260E94E803099000960520DA
:104390000F94C0040D9401960A900C9408950B9507
:1043A0006846FCF731FE002803D0862115A000F0F6
:1043B00047FA07200C900E9401210D950F940CA83C
:1043C000FCF7E8FC002803D092210EA000F038FA98
:1043D000109610A81296FCF767FC002803D0A121C4
:1043E00008A000F02DFA4B208001FCF7B7FF042055
:1043F000FCF7ACFD00221146501EFCF751FC14B036
:1044000070BD00002E2E5C436F6D4C69625C537270
:10441000635C4253502E630013480168012211432C
:1044200001604168114A114041600168104A114021
:1044300001600168012292049143016041683F22BA
:10444000120491434160C16A09090901C162016B0B
:10445000FF22143291430163416B490849004163D3
:104460000021816070470000001002400CB8FF0876
:10447000FFFFF6FE04480169C907C90F02D00121F8
:10448000C9430161704700000010004070B51B4C2B
:10449000E0691B498006C00F11D01A4A0120106044
:1044A000194A10600869401C0861A28C4868401CC9
:1044B0004860174B154D18682A54401C1860E06975
:1044C0000007C00F04D008202062C869401CC861E2
:1044D0002068C006C00F07D0E069C006C00F03D037
:1044E0001020206200F03CF8E0694006C00F03D0C5
:1044F0004020206200F074F870BD000000380140D8
:104500001402002044000020480000203C0300204A
:104510003C00002010B5104CE069E0690007C00FB6
:1045200005D0082020620D48C169491CC16120687E
:10453000C006C00F07D0E069C006C00F03D010202E
:10454000206200F09DF8E0694006C00F03D04020D3
:10455000206200F0E5F810BD00440040A8020020F1
:104560000548416A491C416204490968002901DD86
:104570000121C16770470000140200203C000020A8
:10458000F8B5144D0C46064602212846FDF73CFFBF
:1045900010200090104B324602212846FDF71EFFE6
:1045A000224602212846FDF761FF02212846FDF739
:1045B00037FF0A4804630121417202212846FDF7B2
:1045C0003BFF0548283881688022114381602046DE
:1045D000F8BD00000000024028380140140200200D
:1045E0000248016A491C0162704700001402002061
:1045F00010B50A48407A00280DD1084C206F583475
:10460000002808D12046FCF787F90146E2682068B7
:104610008018FFF7B5FF002010BD00001402002035
:10462000F8B5144D0C46064605212846FDF7ECFE6C
:10463000002000903346104A05212846FDF7CEFEA3
:10464000224605212846FDF711FF05212846FDF7E2
:10465000E7FE0A4844630121817205212846FDF7DF
:10466000EBFE054824388168402211438160002018
:10467000F8BD00000000024024440040A8020020D1
:104680000A480B4900794058802180B2081A09492C
:10469000012208600849CA674A6A521C4A62002817
:1046A00003DD01200549000748607047C453000836
:1046B0000400024040000020A802002000ED00E0BD
:1046C000F8B5144D0C46064604212846FDF79CFE1D
:1046D00010200090104B324604212846FDF77EFE44
:1046E000224604212846FDF7C1FE04212846FDF795
:1046F00097FE0A4804630121417204212846FDF710
:104700009BFE05482838816880221143816020463D
:10471000F8BD00000000024028440040A80200202C
:104720000248016A491C016270470000A80200208B
:1047300010B5054C0A46638821465B1C4380FBF795
:104740003DFF002010BD0000007C000870B50C4645
:104750000B494118002B08D00A4D4519012B03D0F5
:10476000094B9B8A002B00D129468005204603D0A7
:1047700000F042F8002070BDFBF720FFFAE70000D0
:104780000080000800A00008A8140020F8B54188A7
:10479000174A491C4180154901807E2100250A5293
:1047A000ED43802300221146124C002659430C1978
:1047B000314603E0675CFF2F04D1491C9942F9DBC5
:1047C000002E03D0521C082AEDDB00E01546082D10
:1047D00006D208495D436918802200F00DF803E015
:1047E00080220449FBF7EAFE0020F8BDAA5500002C
:1047F000A55A000000C00008F7B50D460646FCF7B4
:10480000EBF902980024870807E0A000325841190C
:1048100000230220FCF7A2F9641CA742F5D80298F5
:104820007C00470807E06000325A4119002301204C
:10483000FCF794F9641CA742F5D8FCF785F9FEBD96
:10484000FEE700000FB410B504A9074B02AA0398B5
:1048500000F028F8044602A9002000F05DFA204686
:1048600010BC08BC04B01847194D000830B4744699
:10487000641E2578641CAB4200D21D46635D5B005C
:10488000E31830BC184702E008C8121F08C1002A0C
:10489000FAD170477047002001E001C1121F002AC1
:1048A000FBD17047FFB591B00F460546002606E0E4
:1048B00025280AD0149A139990476D1C761C2878E5
:1048C0000028F5D1304615B0F0BD00240094012138
:1048D000F34A029400E004436D1C2B780846203B09
:1048E00098401042F7D128782A280ED00221287843
:1048F0000246303A092A15D8009A0A235A43303A18
:1049000080180C436D1C0090F1E701CF0090002847
:1049100005DA012040030443009840420090022041
:1049200004436D1C28782E2815D104200443687890
:104930006D1C2A280AD101CF6D1C02900BE0029950
:104940000A225143303940186D1C029028780146E4
:1049500030390929F3D928786C2810D006DC4C2886
:104960001AD068280ED06A2817D104E0742813D012
:104970007A2812D110E00120400504430CE0012107
:10498000090501E0032109050C436978814203D13F
:104990000120000524186D1C6D1C287803906E28DA
:1049A0001ED00CDC632831D004DC00288AD05828C3
:1049B00011D1B2E064287BD069280CD178E073284B
:1049C0002DD004DC6F2870D0702804D1A7E07528A2
:1049D0006CD078286BD0149A13999047761C62E0BB
:1049E0006002400F022807D003280AD00428386844
:1049F0000AD006603F1D56E03868F1170660416036
:104A0000F8E738680680F5E70670F3E73878694616
:104A100008740020487404A80390012003E038685B
:104A200003900020C0433F1D61070FD5002101E026
:104A30000199491C029A0191914213DA8142F7DBF4
:104A4000019A0399895C0029F2D10BE0002101E071
:104A50000199491C01918142FADB019A0399895C11
:104A60000029F5D101990098139A401A0090214627
:104A7000149B00F03BF901998019461807E0039850
:104A800003990078491C0391149A1399904701984F
:104A9000401E0190401CF2D12146149B139A0098AD
:104AA00000F014F986196D1C09E741E033E034E0A9
:104AB0000A200021049005916002410F022905D0CF
:104AC00001CFC2179446032905D007E0FF1DFF0858
:104AD000FF0003CF06E000B2C2179446042902D1BA
:104AE00040B2C1178C4600226146944506DA0A4658
:104AF0000021404291418C462D2102E0210504D540
:104B00002B216A461176012103E0E10701D0202123
:104B1000F7E7019154E00A200BE0102009E0102093
:104B2000049000210420044308200591029003E032
:104B300008200021059104906002410F022905D050
:104B400001CF00229446032906D006E0FF1DFF088E
:104B5000FF0003CF8C4603E080B2042900D1C0B22D
:104B60000021019121072BD50399702906D0049AC1
:104B70001021059B4A401A4305D00EE040216A46A9
:104B80001176012108E06146014306D030216A46D2
:104B900011760399517602210191049A0821059B0F
:104BA0004A401A430CD16146014301D1610707D540
:104BB00030216A461176012101910299491E029124
:104BC0000399582904D037A103910FA90F910DE043
:104BD00039A1F9E76146059B049AFBF714FB039B97
:104BE0008C469B5C0F9A521E0F92137061460143D4
:104BF000F0D10F9807A9081A20300390600704D558
:104C0000012000048443029801E0012002900399EE
:104C1000884201DD401A00E000204118029001980E
:104C200009180098401A0090E00306D42146149B0E
:104C3000139A009800F05AF886190020049008E0B2
:104C400006A9085C149A139990470498401C761C96
:104C5000049001998842F3DBE0030CD52146149BB4
:104C6000139A009800F042F8861904E0149A302054
:104C700013999047761C0299481E02900029F5DC92
:104C800008E00F980F990078491C0F91149A139916
:104C90009047761C0399481E03900029F1DCFBE63F
:104CA0000928010030313233343536373839616202
:104CB00063646566000000003031323334353637C6
:104CC000383941424344454600000000F8B50446E7
:104CD00000251E461746880404D405E039462020E6
:104CE000B0476D1C641EF9D52846F8BDFFB50446D3
:104CF000002581B01E46C80301D5302700E02027DB
:104D0000880404D505E038460399B0476D1C641E3D
:104D1000F9D5284605B0F0BD0A68531C0B60107029
:104D20007047000010B50A2101A0FEF7E1FE10BD9A
:104D30001B5B324A1B5B303B3048000030B50346FA
:104D40000B48002900D101210A4C491E0ED31A78C4
:104D500050400022C50702D04008604000E04008F3
:104D6000521CD2B2082AF5D35B1CEEE730BD00001E
:104D7000FFFF000001A0000070B50A4DFF23EE1DEB
:104D80001A46F93605E0047854402A5D5A40335DEE
:104D9000401C0C46491E89B2002CF4D11802104365
:104DA00070BD0000CA55000870B504460C480022CA
:104DB0000C4E11E02378521C1D4645402D07ED0E88
:104DC000755B00094540180968400007C00E305A5D
:104DD0002B09584092B2641C8A42EBD370BD00008C
:104DE000FFFF0000CA57000810B5084A084B07E04B
:104DF000047854402406E40D1C5B120A6240401CF7
:104E0000491EF5D2D04380B210BD0000FFFF000064
:104E1000CA53000806C00021016041608160C16082
:104E2000012202614161084670470000074910B540
:104E30004A8D0B464C3BD054488D401C80B248856F
:104E4000642801D35120488510BD0000741400204F
:104E5000F94F88B00126FF203E830530F74B8022B2
:104E60000090991AF648FCF7BCF84020F54B024632
:104E7000191A0090F448FCF7B4F8FBF7CDFE0021B6
:104E8000F24A0D4660204843801845608560056100
:104E900045618561C561056285624562C562491CDF
:104EA00005630929EEDBEA4CEA482567C06A6066BB
:104EB000E9480068A066E948406AE066FFF75AFAE8
:104EC000E849E7480860FCF7A7FAFDF7F9FCFDF7A9
:104ED000E3FCFDF727FAE448FEF79EFED64806837A
:104EE000FEF792FE1021A06308430107090F6063DB
:104EF000DE4AC006DE48117003D50670DD48057035
:104F000002E00570DB480670DB480170FBF700FC2F
:104F1000D64801270178D8480170D848D849077089
:104F2000E12080020860FDF70FFEFDF79FFEFDF710
:104F30007BFDD4484168402631434160FDF75AFD6E
:104F4000FDF7D8FDD048016839430160CF480168BA
:104F50002022114301600168102739430160016874
:104F6000314301608021CA48FFF75AFBC9480168F4
:104F7000394301600168314301600A20FBF786FD77
:104F80000120FFF745F80020FFF72AF80020FFF77F
:104F900033F8FFF7ADF8FBF763FDA74E6066358287
:104FA0007582B148C0883082308A01280AD1FCF766
:104FB000EDF9208F202108407082708A002801D0EE
:104FC000FFF758F9B4485A210790B44F4184B44DC3
:104FD00000262E7001206870FBF742FD2861FBF768
:104FE0000DFE0690FEF710FE05469348008AC007A6
:104FF0000BD0A806208F04D5800606D4FFF73AF917
:1050000003E0800601D5FFF76DF9A5630698E0631C
:105010000920C0060069B884A2480069F884A24843
:1050200000693885A14800697885FBF795FBFBF797
:1050300017FD9B4D68619E480068002801D00798C5
:105040008682206CC006C00E02281CD1FBF72EF908
:105050009748016800290ED007998E8295490A6801
:10506000002A10D1006808609348006893490860DE
:10507000FEF7B4F907E08F490A68002A03D00068F8
:105080000860FEF7C3F96C48008A01280BD16A4812
:10509000818A00291FD08A49A960C18A8948016094
:1050A000A868FEF7BBF9606E69696166081AA066B8
:1050B000E16E884200D2E066216F884200D9206705
:1050C000FBF7CEFCA8616A480078002818D07E491A
:1050D00000200B780BE07D49DEE77D49132209189B
:1050E000520189180A7D7B4909184A70401C984270
:1050F000F3DB61480078002802D00220FCF784FA34
:105100000698800402D50120287000E02E700698D1
:10511000000502D50120687000E06E7055480078E7
:1051200000281AD00220FCF74BFC606C002801D14B
:105130006948067068480178079881866749086859
:10514000800402D50120287000E02E700868000558
:1051500002D50120687000E06E70606C002801D0FC
:10516000401E6064A06C002801D0401EA06432483C
:10517000018B00293FD06878FEF74AFF6878FEF778
:105180002FFF6878FEF720FF6878002801D1012002
:1051900000E00020FEF730FFFBF762FCE861FBF760
:1051A0005FFC2862FBF75CFC0A2168620846FAF79C
:1051B0008BFF0020401C4028FCDB206C4849401C31
:1051C00020640868002836DD1D4AD26F002A32D0DC
:1051D00082B244490120FDF711FE002805D0404865
:1051E000404902680120FCF70DFD3D480660144867
:1051F000C6676E608EE0008A01280FD0606C0028C0
:1052000010D06878FEF704FFA06C00280CD06878F6
:10521000FEF7E6FE6878FEF7D7FEBAE73248006888
:105220000028EFD02878EDE70020FEF7D9FE002017
:10523000FEF7CAFEABE759E0A8140020A81500202D
:1052400014020020EC160020A80200205C050020BB
:105250007412002080F7FF1F300000200010024071
:105260001027000014000020740C002050000020C3
:105270004C0000204D00002057000020510000206D
:105280003400002000300140001000400038014090
:10529000BC03002000440040340F002074140020A0
:1052A000E40000200004004800080048000C00480A
:1052B000BC000020C000002018000020C400002016
:1052C00000A0000894000020CB000020008000080F
:1052D000F40C00204C0400203C0400206800002056
:1052E0003C0000203C0300206C0A0020284968682C
:1052F00088420DD9274841680122120511434160B7
:105300004168520003235B0599431143416001E06A
:10531000401C686020480078002802D00020FBF77D
:10532000B5FB18221D496846FAF73FFF1C4D0020C7
:105330006E461C494200511840310A891105130B71
:105340001207090E120F002918D0002B02D0012BD2
:1053500006D013E0144B591809239B01C91804E027
:10536000114B5B18132149015918C97C0123934043
:10537000194203D081007158A96102E0810071587F
:10538000A962401C0628D4DB0949084808601EE6CB
:10539000C0270900003801404D000020A058000837
:1053A00000040048740C0020F40C0020AAAA00009D
:1053B00000300040112233445566778899AABBCC4F
:1053C000DDEEFF00081C3044580000008911122354
:1053D0009B322446AD573665BF74488CC19D5AAF89
:1053E000D3BE6CCAE5DB7EE9F7F881100801933380
:1053F0001A22A5562C47B7753E64C99C408DDBBF69
:1054000052AEEDDA64CBFFF976E802218B30100260
:1054100099132667AF763444BD554AADC3BC588E48
:10542000D19F6EEBE7FA7CC8F5D983310A2091123F
:105430001803A7772E66B5543C45CBBD42ACD99E28
:10544000508FEFFB66EAFDD874C904428D53166194
:105450009F702004A9153227BB364CCEC5DF5EED08
:10546000D7FC6888E1997AABF3BA85520C439771FF
:105470001E60A1142805B3373A26CDDE44CFDFFDE8
:1054800056ECE9986089FBBB72AA06638F721440E0
:105490009D512225AB343006B9174EEFC7FE5CCCC8
:1054A000D5DD6AA9E3B8788AF19B87730E629550BF
:1054B0001C41A3352A24B1163807CFFF46EEDDDCA8
:1054C00054CDEBB962A8F99A708B088481951AA71C
:1054D00093B62CC2A5D33EE1B7F04008C919522BB0
:1054E000DB3A644EED5F766DFF7C899400859BB757
:1054F00012A6ADD224C3BFF136E0C1184809D33B90
:105500005A2AE55E6C4FF77D7E6C0AA583B4188637
:1055100091972EE3A7F23CC0B5D14229CB38500A6F
:10552000D91B666FEF7E744CFD5D8BB502A4999616
:105530001087AFF326E2BDD034C1C3394A28D11A4F
:10554000580BE77F6E6EF55C7C4D0CC685D71EE56B
:1055500097F42880A1913AA3B3B2444ACD5B56692F
:10556000DF78600CE91D722FFB3E8DD604C79FF5D6
:1055700016E4A9902081BBB332A2C55A4C4BD7790F
:105580005E68E11C680DF33F7A2E0EE787F61CC4B7
:1055900095D52AA1A3B03882B193466BCF7A5448EF
:1055A000DD59622DEB3C700EF91F8FF706E69DD496
:1055B00014C5ABB122A0B9923083C77B4E6AD558CF
:1055C0005C49E33D6A2CF11E780F00C1814001C0A7
:1055D000804101C0804100C1814001C0804100C1C3
:1055E000814000C1814001C0804101C0804100C1B3
:1055F000814000C1814001C0804100C1814001C0A3
:10560000804101C0804100C1814001C0804100C192
:10561000814000C1814001C0804100C1814001C082
:10562000804101C0804100C1814000C1814001C072
:10563000804101C0804100C1814001C0804100C162
:10564000814000C1814001C0804101C0804100C152
:10565000814000C1814001C0804100C1814001C042
:10566000804101C0804100C1814000C1814001C032
:10567000804101C0804100C1814001C0804100C122
:10568000814000C1814001C0804100C1814001C012
:10569000804101C0804100C1814001C0804100C102
:1056A000814000C1814001C0804101C0804100C1F2
:1056B000814000C1814001C0804100C1814001C0E2
:1056C000804101C0804100C1814000C0C101C303CD
:1056D00002C2C60607C705C5C404CC0C0DCD0FCF4A
:1056E000CE0E0ACACB0BC90908C8D81819D91BDBBA
:1056F000DA1A1EDEDF1FDD1D1CDC14D4D515D7170A
:1057000016D6D21213D311D1D010F03031F133F3B9
:10571000F23236F6F737F53534F43CFCFD3DFF3F09
:105720003EFEFA3A3BFB39F9F83828E8E929EB2B39
:105730002AEAEE2E2FEF2DEDEC2CE42425E527E7C9
:10574000E62622E2E323E12120E0A06061A163A339
:10575000A26266A6A767A56564A46CACAD6DAF6FC9
:105760006EAEAA6A6BAB69A9A86878B8B979BB7B39
:105770007ABABE7E7FBF7DBDBC7CB47475B577B789
:10578000B67672B2B373B17170B0509091519353B9
:10579000529296565797559594549C5C5D9D5F9F89
:1057A0009E5E5A9A9B5B99595898884849894B8BB9
:1057B0008A4A4E8E8F4F8D4D4C8C44848545874749
:1057C00046868242438341818040000001CC01D85B
:1057D000001401F0003C002801E401A0006C0078F6
:1057E00001B40050019C01880044030E0401000133
:1057F000000104010006000000000000000000009D
:1058000006000000AA550000000100000000000092
:10581000010001000009000000000000000002007B
:10582000000000090000000000000000000000006F
:105830000000000000000000000000001010101028
:105840001010101010101010101010101000200068
:105850003000400050006000030000000400000021
:10586000050000000600000007000000080000001E
:10587000090000000A0000000B0000000C000000FE
:105880001100A55AAA550000000000000000000009
:1058900000000000081C304458081C304458000028
:1058A00000040000000800000010000000200000BC
:1058B0000040000000800000000000000000000028
:1058C00001020304060708090000000001020304A6
:1058D000F05800080000002014010000864800086D
:1058E000045A0008140100203C1A000096480008E1
:1058F00000000000000000000000000000000000A8
:10590000010000001027000000000000000000005F
:105910000000000000000000000000000000000087
:10592000000000000084030040420F00000000005F
:105930000000000000000000000000000000010066
:105940000000000101010000000000000000000054
:105950000000000000000000000000000000000047
:105960000000000000000000000000000000000037
:105970000000000001000000000000000000000026
:105980000100000097000000FFFFFFFF0000000083
:105990000000000000000000000000000000000007
:1059A00000000000000000000000000000000000F7
:1059B00000000000000000000000080800000000D7
:1059C00000000000000000000000000000000000D7
:1059D000000000000000000000000000008000083F
:1059E00000000000000000000000000000000000B7
:1059F000000000000000000000000000001BB700D5
:045A000000000000A2
:04000005080000B53A
:00000001FF
